:020000040000FA
:09000000020A560220032222220A
:03000B0002200BC5
:03001300022013B5
:03001B0002201BA5
:0300230002202395
:03002B0002202B85
:0300330002203375
:03003B0002203B65
:0300430002204355
:03004B0002204B45
:0300530002205335
:03005B0002205B25
:0300630002206315
:03006B0002206B05
:03007300022073F5
:03007B0002207BE5
:03008300022083D5
:03008B0002208BC5
:03009300022093B5
:03009B0002209BA5
:0300A3000220A395
:0300AB000220AB85
:1000B3000220B3E590540C23C0E0740DC0E0C0826D
:1000C300C083020D00E590540C23C0E0740DC0E022
:1000D300C082C083020D08E590540C23C0E0740D68
:1000E300C0E0C082C083020D10E590540C23C0E031
:1000F300740DC0E0C082C083020D18EFC403900DDD
:02010300007387
:10010600E56A245EF8E6056A22785B300702785EC7
:10011600E475F0011208B90208242000EB7F2ED204
:10012600008018EF540F2490D43440D4FF30040BD1
:10013600EF24BFB41A0050032461FFE56B6002157B
:100146006B056EE56E7002056D30070D785BE47524
:10015600F0011208B9EF0208A7020C927403D20745
:100166008003E4C207F56A8B5B8A5C895DE4F56B04
:10017600F56DF56EE56B60077F2012014180F57520
:100186006CFFC201C200C202C203C205C206C20897
:1001960012010FFF700D3007057F00120152AF6E7E
:1001A600AE6D22B4255FC2D5C20412010FFF24D062
:1001B600B40A00501A75F00A786B30D50508B6FFF8
:1001C6000106C6A426F620D5047002D20380D924DF
:1001D600CFB41A00EF5004C2E5D204020352D20192
:1001E60080C6D20080C0D20280BCD2D580BAD205E9
:1001F60080B47F201201412002077401B56B0040D4
:10020600F1120106FF12014102017AD208D20680DC
:1002160095120106FB120106FA120106F94A4B7005
:100226000679237A047BFF20022EE56B602A7E0086
:100236008E8275830012087A60060EEE656C70F089
:10024600C2D5EBC0E0EAC0E0E9C0E0EE120399D007
:10025600E0F9D0E0FAD0E0FB120824FF60AAEBC078
:10026600E0EAC0E0E9C0E0120141D0E02401F9D0A3
:10027600E03400FAD0E0FBE56C0460DCD56CD98094
:10028600877BFF7A037995D202809C791080027968
:1002960008C206C2088008D2D5790A8004790AC243
:1002A600D5E56C047002F56CE4FAFDFEFF1201065A
:1002B600FC7B08200113120106FD7B1030000A1298
:1002C6000106FE120106FF7B20EC3382D592D55043
:1002D60013C3E43000069FFFE49EFEE42001039D65
:1002E600FDE49CFCE4CBF8C201EC700CCFCECDCC87
:1002F600E824F8F870F38017C3EF33FFEE33FEED12
:1003060033FDEC33FCEB33FB994002FB0FD8E9EBF2
:10031600300105F8D0E0C448B201C0E00AEC4D4E09
:100326004F78207B0070C2EAB56C0040BCC0E0127A
:10033600039BD0F0D0E0200104C4C0E0C4B201C0E9
:10034600F012012AD0F0D5F0EB02017A1208C902A8
:10035600175302915801E84C01E44202954F029D61
:1003660044029D4901FD4302A35502874602874583
:1003760002874704435001EC2D01F02E02132B0196
:10038600F423021120042C2A01AC480000020B3F82
:100396003F3F00790AA2D5200314300509B910029F
:1003A6000404B9080104A2D5200602500104200263
:1003B600689202B56B005034C0E07F203003197F8D
:1003C60030A20272067205500F1203F2C202C20672
:1003D600C205C2087F30800F300503E9C0E0120174
:1003E60041300503D0E0F9D0E0B56BCC3005177F7E
:1003F60030B9100C1201417F583004077F78800312
:10040600B908031201413002057F2D0201417F2008
:100416002008F87F2B2006F322920280CF286E75E3
:100426006C6C2900D2011201063001F8C201786B0A
:1004360030D50108F60201AC2D5043495812010689
:100446002403B405004001E490043E931201327483
:100456003A120132D203756B04020291E4F556F5A5
:1004660057F558120C818F31BF3BF8120C118F4B88
:10047600120C11E48F50F54FF54EF54DAE4FAD4EC3
:10048600AC4D78081208618F508E4F8D4E8C4D12F0
:100496000C11E5504FF550E54FF54FE54EF54EE59D
:1004A6004DF54D120C118F4CE4F52FF530C3E530A8
:1004B600954BE52F94005014120C1174322530F828
:1004C600A6070530E53070E5052F80E1120C118F87
:1004D60055E4FF7E20FDFCAB50AA4FA94EA84DC3A4
:1004E60012083D5003020587D3E54C9401748094AD
:1004F6008040030205877B007A00793275620085A9
:100506004B63AF50AE4FAD4EAC4D120AE8E4F55614
:10051600F52FF530C3E530954BE52F94005024E5D3
:10052600302550FFE52F354FFEE4354EFDE4354DC1
:10053600FC1208EFEF2556F5560530E53070D50567
:100546002F80D1E54B2556F556AF50AE4FAD4EAC8C
:100556004D780812084EEF2556F556E550FFEF2563
:1005660056F556254CF5562555F556FF3395E04F6D
:10057600600F1200077BFF7A0C79D5120168020022
:10058600081200077BFF7A0C79DF12016812000857
:10059600E54C64016003020469F52FF5300530E58A
:1005A600307002052FB410F5E52FB427F075080159
:1005B600E4F557F558F554755320F552F551E47F97
:1005C600FE7EFFFDFCAB54AA53A952A851C31208E4
:1005D6003D502CAF54AE53AD52AC511208EFEF253F
:1005E60058F558E43557F557E5542401F554E435E4
:1005F60053F553E43552F552E43551F55180BFC3F6
:10060600E49558F55AE49557F559FF3395E08F6C04
:100616007FFE7EFF7D007C00120630855A6C7FFFD0
:100626007EFF7D007C00120630228F6B8E6A8D69FC
:100636008C6885A76DA2AF920085F56EC2AFE4F512
:10064600A7FF7E80FDFCAB6BAA6AA969A868C312E6
:10065600083D500B856A6F856B7053F5CF8076E445
:10066600FFFE7D01FCAB6BAA6AA969A868C31208E4
:100676003D5020E56BF56BE56A4480F56AE569F562
:1006860069E568F568856A6F856B7053F5CF43F544
:100696001080427F007E807D017C00AB6BAA6AA938
:1006A60069A868C312083D5020E56BF56BE56A44FE
:1006B60080F56AE569F569E568F568856A6F856BB1
:1006C6007053F5CF43F520800C856A6F856B7053A8
:1006D600F5CF43F530E4F5EF75FFA0FFEFC394FFC8
:1006E6007480948050030F80F3E5FF20E6037F00BB
:1006F6002275EF0275B7A575B7F1438F0175FFA097
:1007060075EF02857082856F83E56CF0E4F5EF7511
:10071600FF8075EF02538FFE856EF5856DA7A200EB
:1007260092AF7F01228F368E358D348C3385A73775
:10073600A2AF920085F538C2AFE4F5A7FF7E80FD33
:10074600FCAB36AA35A934A833C312083D500B8535
:10075600353985363A53F5CF8076E4FFFE7D01FCC8
:10076600AB36AA35A934A833C312083D5020E53666
:10077600F536E5354480F535E534F534E533F533BE
:1007860085353985363A53F5CF43F51080427F00DB
:100796007E807D017C00AB36AA35A934A833C3120E
:1007A600083D5020E536F536E5354480F535E53427
:1007B600F534E533F53385353985363A53F5CF4388
:1007C600F520800C85353985363A53F5CF43F5301B
:1007D600E4F5EF75FFA0FFEFC394FF74809480509B
:1007E600030F80F3E5FF20E6037F002275EF027515
:1007F600B7A575B7F1438F0375FFA075EF02853A6C
:1008060082853983E4F0F5EF75FF8075EF02538F2B
:10081600FC8538F58537A7A20092AF7F0122BB0180
:100826000689828A83E0225002E722BBFE02E32287
:1008360089828A83E49322EB9FF5F0EA9E42F0E9EF
:100846009D42F0E89C45F022E8600FECC313FCEDF6
:1008560013FDEE13FEEF13FFD8F122E8600FEFC38E
:1008660033FFEE33FEED33FDEC33FCD8F1228A8301
:100876008982E473BB010CE58229F582E5833AF5AA
:1008860083E0225006E92582F8E622BBFE06E9252A
:1008960082F8E222E58229F582E5833AF583E4933C
:1008A60022BB010689828A83F0225002F722BBFE10
:1008B60001F322FAE6FB0808E6F925F0F618E6CA7F
:1008C6003AF622D083D082F8E493701274019370C2
:1008D6000DA3A393F8740193F5828883E4737402DD
:1008E600936860EFA3A3A380DF8F5E8E5D8D5C8C23
:1008F6005B85A75FA2AF920085F560C2AFE4F5A75E
:10090600FF7E80FDFCAB5EAA5DA95CA85BC31208F6
:100916003D500B855D61855E6253F5CF8076E4FFC1
:10092600FE7D01FCAB5EAA5DA95CA85BC312083D17
:100936005020E55EF55EE55D4480F55DE55CF55CC1
:10094600E55BF55B855D61855E6253F5CF43F5102A
:1009560080427F007E807D017C00AB5EAA5DA95C43
:10096600A85BC312083D5020E55EF55EE55D448058
:10097600F55DE55CF55CE55BF55B855D61855E6275
:1009860053F5CF43F520800C855D61855E6253F596
:10099600CF43F530856282856183E493FF8560F5F8
:1009A600855FA7A20092AF2285EF26E4F5A753D96B
:1009B600BF120CA1120C32C2AF752BFF752C20F59D
:1009C6002DF522F523F52A752920F528F527E47F4C
:1009D600FE7EFFFDFCAB2AAA29A928A827C3120878
:1009E6003D502CAF2AAE29AD28AC271208EFEF25D3
:1009F60023F523E43522F522E52A2401F52AE435F8
:100A060029F529E43528F528E43527F52780BF7F21
:100A1600FE7EFF7D007C001208EFEF752500F524B1
:100A26007FFF7EFF7D007C001208EFEF2525F52570
:100A3600E43524F524E5252523F523E5243522F59B
:100A46002245236003020BB0AA2CA92D120874229A
:100A5600120006787FE4F6D8FD758170120D00024B
:100A66000AA30209AEE493A3F8E493A34003F68035
:100A760001F208DFF48029E493A3F85407240CC894
:100A8600C333C4540F4420C8834004F4568001463F
:100A9600F6DFE4800B0102040810204080900CACC5
:100AA600E47E019360BCA3FF543F30E509541FFE6A
:100AB600E493A360010ECF54C025E060A840B8E4DB
:100AC60093A3FAE493A3F8E493A3C8C582C8CAC55E
:100AD60083CAF0A3C8C582C8CAC583CADFE9DEE7F0
:100AE60080BE8F5E8E5D8D5C8C5B8B5F8A6089615C
:100AF6008F678E668D658C64E563255EFFE56235DE
:100B06005DFEE4355CFDE4355BFCAB67AA66A96572
:100B1600A864C312083D5035AF67AE66AD65AC64D8
:100B2600AB5F0561E561AA607002056014F9120801
:100B360024F56C120630E5672401F567E43566F5A1
:100B460066E43565F565E43564F56480AB22E4F565
:100B560032753120F530F52FE47FFF7EFFFDFCABCB
:100B660032AA31A930A82FC312083D5022AF32AEA7
:100B760031AD30AC2F12072BE42532F532E5313496
:100B860002F531E43530F530E4352FF52F80C9E430
:100B96002532FFE5313402FEE43530FDE4352FFC25
:100BA60012072BE4F50875090122120C6A7F01125F
:100BB6000C4F120C818F2EE52E24CE601404701D6E
:100BC6007BFF7A0C79B3120168120B54120462800F
:100BD6000C7BFF7A0C79BC12016875EF10120C8140
:100BE6008F2E80D3EF7E0024D0B40A00401B24F958
:100BF600B40A004011B41000400F24E0B40A0040CB
:100C060005B41000400374FFFEFF22120C818F5CB6
:100C1600120C818F5DAF5C120BEAEFC454F0F55BEA
:100C2600AF5D120BEAEF255BF55BFF22AFA775A759
:100C36000F75A41075A50375A61F75AE0F75AFFFCA
:100C460075E10175C7C08FA722D2B0D2B1D2B2D298
:100C5600B3D290D291C2A0D2A4EF24FF92A1D2A384
:100C660075B5FF22AFA7E4F5A775981075A70F75A0
:100C7600ACD875ADFF75AB438FA722AFA7E4F5A738
:100C86003098FDAE99C2988FA7AF0622AEA7E4F5BD
:100C9600A78F993099FDC2998EA722AFA775A70F86
:100CA60075A1C78FA72201090001080000457261DE
:100CB60073696E67000052455345540000312E4556
:100CC600726173650A00322E5265736574000063A3
:100CD60072635F6661696C00006F6B5F777269743F
:030CE600650000A6
:040D00005390F322F7
:070D080043900C5390F72209
:070D100043900C5390FB22FD
:040D180043900C22D6
:00000001FF
